
D:\STM32\Program\1.11_Odchudzanie\um0427\FWLib\project\RIDE\STM3210E-EVAL\stm32f10x_adc.o:     file format elf32-littlearm
D:\STM32\Program\1.11_Odchudzanie\um0427\FWLib\project\RIDE\STM3210E-EVAL\stm32f10x_adc.o

Disassembly of section .text.ADC_Init:

00000000 <ADC_Init>:
ADC_Init():
D:\STM32\Program\1.11_Odchudzanie\um0427\FWLib\library\src/stm32f10x_adc.c:190
   0:	6843      	ldr	r3, [r0, #4]
D:\STM32\Program\1.11_Odchudzanie\um0427\FWLib\library\src/stm32f10x_adc.c:196
   2:	680a      	ldr	r2, [r1, #0]
   4:	f423 2370 	bic.w	r3, r3, #983040	; 0xf0000
   8:	f423 7380 	bic.w	r3, r3, #256	; 0x100
   c:	4313      	orrs	r3, r2
   e:	790a      	ldrb	r2, [r1, #4]
D:\STM32\Program\1.11_Odchudzanie\um0427\FWLib\library\src/stm32f10x_adc.c:175
  10:	b510      	push	{r4, lr}
D:\STM32\Program\1.11_Odchudzanie\um0427\FWLib\library\src/stm32f10x_adc.c:196
  12:	ea43 2302 	orr.w	r3, r3, r2, lsl #8
D:\STM32\Program\1.11_Odchudzanie\um0427\FWLib\library\src/stm32f10x_adc.c:198
  16:	6043      	str	r3, [r0, #4]
D:\STM32\Program\1.11_Odchudzanie\um0427\FWLib\library\src/stm32f10x_adc.c:209
  18:	68cb      	ldr	r3, [r1, #12]
  1a:	688a      	ldr	r2, [r1, #8]
D:\STM32\Program\1.11_Odchudzanie\um0427\FWLib\library\src/stm32f10x_adc.c:202
  1c:	6884      	ldr	r4, [r0, #8]
D:\STM32\Program\1.11_Odchudzanie\um0427\FWLib\library\src/stm32f10x_adc.c:209
  1e:	431a      	orrs	r2, r3
  20:	4b08      	ldr	r3, [pc, #32]	(44 <ADC_Init+0x44>)
  22:	ea04 0303 	and.w	r3, r4, r3
  26:	431a      	orrs	r2, r3
  28:	794b      	ldrb	r3, [r1, #5]
  2a:	ea42 0243 	orr.w	r2, r2, r3, lsl #1
D:\STM32\Program\1.11_Odchudzanie\um0427\FWLib\library\src/stm32f10x_adc.c:212
  2e:	6082      	str	r2, [r0, #8]
D:\STM32\Program\1.11_Odchudzanie\um0427\FWLib\library\src/stm32f10x_adc.c:222
  30:	7c0b      	ldrb	r3, [r1, #16]
D:\STM32\Program\1.11_Odchudzanie\um0427\FWLib\library\src/stm32f10x_adc.c:216
  32:	6ac2      	ldr	r2, [r0, #44]
D:\STM32\Program\1.11_Odchudzanie\um0427\FWLib\library\src/stm32f10x_adc.c:222
  34:	3b01      	subs	r3, #1
D:\STM32\Program\1.11_Odchudzanie\um0427\FWLib\library\src/stm32f10x_adc.c:218
  36:	f422 0270 	bic.w	r2, r2, #15728640	; 0xf00000
D:\STM32\Program\1.11_Odchudzanie\um0427\FWLib\library\src/stm32f10x_adc.c:222
  3a:	b2db      	uxtb	r3, r3
  3c:	ea42 5203 	orr.w	r2, r2, r3, lsl #20
D:\STM32\Program\1.11_Odchudzanie\um0427\FWLib\library\src/stm32f10x_adc.c:224
  40:	62c2      	str	r2, [r0, #44]
D:\STM32\Program\1.11_Odchudzanie\um0427\FWLib\library\src/stm32f10x_adc.c:225
  42:	bd10      	pop	{r4, pc}
  44:	fff1f7fd 	.word	0xfff1f7fd
Disassembly of section .text.ADC_StructInit:

00000000 <ADC_StructInit>:
ADC_StructInit():
D:\STM32\Program\1.11_Odchudzanie\um0427\FWLib\library\src/stm32f10x_adc.c:239
   0:	2300      	movs	r3, #0
   2:	6003      	str	r3, [r0, #0]
D:\STM32\Program\1.11_Odchudzanie\um0427\FWLib\library\src/stm32f10x_adc.c:242
   4:	7103      	strb	r3, [r0, #4]
D:\STM32\Program\1.11_Odchudzanie\um0427\FWLib\library\src/stm32f10x_adc.c:245
   6:	7143      	strb	r3, [r0, #5]
D:\STM32\Program\1.11_Odchudzanie\um0427\FWLib\library\src/stm32f10x_adc.c:248
   8:	6083      	str	r3, [r0, #8]
D:\STM32\Program\1.11_Odchudzanie\um0427\FWLib\library\src/stm32f10x_adc.c:251
   a:	60c3      	str	r3, [r0, #12]
D:\STM32\Program\1.11_Odchudzanie\um0427\FWLib\library\src/stm32f10x_adc.c:254
   c:	3301      	adds	r3, #1
   e:	7403      	strb	r3, [r0, #16]
D:\STM32\Program\1.11_Odchudzanie\um0427\FWLib\library\src/stm32f10x_adc.c:255
  10:	4770      	bx	lr
  12:	46c0      	nop			(mov r8, r8)
Disassembly of section .text.ADC_Cmd:

00000000 <ADC_Cmd>:
ADC_Cmd():
D:\STM32\Program\1.11_Odchudzanie\um0427\FWLib\library\src/stm32f10x_adc.c:272
   0:	b119      	cbz	r1, a <ADC_Cmd+0xa>
D:\STM32\Program\1.11_Odchudzanie\um0427\FWLib\library\src/stm32f10x_adc.c:275
   2:	6883      	ldr	r3, [r0, #8]
   4:	f043 0301 	orr.w	r3, r3, #1	; 0x1
   8:	e002      	b.n	10 <ADC_Cmd+0x10>
D:\STM32\Program\1.11_Odchudzanie\um0427\FWLib\library\src/stm32f10x_adc.c:280
   a:	6883      	ldr	r3, [r0, #8]
   c:	f023 0301 	bic.w	r3, r3, #1	; 0x1
  10:	6083      	str	r3, [r0, #8]
D:\STM32\Program\1.11_Odchudzanie\um0427\FWLib\library\src/stm32f10x_adc.c:282
  12:	4770      	bx	lr
Disassembly of section .text.ADC_DMACmd:

00000000 <ADC_DMACmd>:
ADC_DMACmd():
D:\STM32\Program\1.11_Odchudzanie\um0427\FWLib\library\src/stm32f10x_adc.c:300
   0:	b119      	cbz	r1, a <ADC_DMACmd+0xa>
D:\STM32\Program\1.11_Odchudzanie\um0427\FWLib\library\src/stm32f10x_adc.c:303
   2:	6883      	ldr	r3, [r0, #8]
   4:	f443 7380 	orr.w	r3, r3, #256	; 0x100
   8:	e002      	b.n	10 <ADC_DMACmd+0x10>
D:\STM32\Program\1.11_Odchudzanie\um0427\FWLib\library\src/stm32f10x_adc.c:308
   a:	6883      	ldr	r3, [r0, #8]
   c:	f423 7380 	bic.w	r3, r3, #256	; 0x100
  10:	6083      	str	r3, [r0, #8]
D:\STM32\Program\1.11_Odchudzanie\um0427\FWLib\library\src/stm32f10x_adc.c:310
  12:	4770      	bx	lr
Disassembly of section .text.ADC_ITConfig:

00000000 <ADC_ITConfig>:
ADC_ITConfig():
D:\STM32\Program\1.11_Odchudzanie\um0427\FWLib\library\src/stm32f10x_adc.c:337
   0:	b2c9      	uxtb	r1, r1
D:\STM32\Program\1.11_Odchudzanie\um0427\FWLib\library\src/stm32f10x_adc.c:339
   2:	b11a      	cbz	r2, c <ADC_ITConfig+0xc>
D:\STM32\Program\1.11_Odchudzanie\um0427\FWLib\library\src/stm32f10x_adc.c:342
   4:	6843      	ldr	r3, [r0, #4]
   6:	ea41 0303 	orr.w	r3, r1, r3
   a:	e002      	b.n	12 <ADC_ITConfig+0x12>
D:\STM32\Program\1.11_Odchudzanie\um0427\FWLib\library\src/stm32f10x_adc.c:347
   c:	6843      	ldr	r3, [r0, #4]
   e:	ea23 0301 	bic.w	r3, r3, r1
  12:	6043      	str	r3, [r0, #4]
D:\STM32\Program\1.11_Odchudzanie\um0427\FWLib\library\src/stm32f10x_adc.c:349
  14:	4770      	bx	lr
  16:	46c0      	nop			(mov r8, r8)
Disassembly of section .text.ADC_ResetCalibration:

00000000 <ADC_ResetCalibration>:
ADC_ResetCalibration():
D:\STM32\Program\1.11_Odchudzanie\um0427\FWLib\library\src/stm32f10x_adc.c:364
   0:	6883      	ldr	r3, [r0, #8]
   2:	f043 0308 	orr.w	r3, r3, #8	; 0x8
   6:	6083      	str	r3, [r0, #8]
D:\STM32\Program\1.11_Odchudzanie\um0427\FWLib\library\src/stm32f10x_adc.c:365
   8:	4770      	bx	lr
   a:	46c0      	nop			(mov r8, r8)
Disassembly of section .text.ADC_GetResetCalibrationStatus:

00000000 <ADC_GetResetCalibrationStatus>:
ADC_GetResetCalibrationStatus():
D:\STM32\Program\1.11_Odchudzanie\um0427\FWLib\library\src/stm32f10x_adc.c:382
   0:	6880      	ldr	r0, [r0, #8]
D:\STM32\Program\1.11_Odchudzanie\um0427\FWLib\library\src/stm32f10x_adc.c:395
   2:	f3c0 00c0 	ubfx	r0, r0, #3, #1
   6:	4770      	bx	lr
Disassembly of section .text.ADC_StartCalibration:

00000000 <ADC_StartCalibration>:
ADC_StartCalibration():
D:\STM32\Program\1.11_Odchudzanie\um0427\FWLib\library\src/stm32f10x_adc.c:410
   0:	6883      	ldr	r3, [r0, #8]
   2:	f043 0304 	orr.w	r3, r3, #4	; 0x4
   6:	6083      	str	r3, [r0, #8]
D:\STM32\Program\1.11_Odchudzanie\um0427\FWLib\library\src/stm32f10x_adc.c:411
   8:	4770      	bx	lr
   a:	46c0      	nop			(mov r8, r8)
Disassembly of section .text.ADC_GetCalibrationStatus:

00000000 <ADC_GetCalibrationStatus>:
ADC_GetCalibrationStatus():
D:\STM32\Program\1.11_Odchudzanie\um0427\FWLib\library\src/stm32f10x_adc.c:428
   0:	6880      	ldr	r0, [r0, #8]
D:\STM32\Program\1.11_Odchudzanie\um0427\FWLib\library\src/stm32f10x_adc.c:441
   2:	f3c0 0080 	ubfx	r0, r0, #2, #1
   6:	4770      	bx	lr
Disassembly of section .text.ADC_SoftwareStartConvCmd:

00000000 <ADC_SoftwareStartConvCmd>:
ADC_SoftwareStartConvCmd():
D:\STM32\Program\1.11_Odchudzanie\um0427\FWLib\library\src/stm32f10x_adc.c:458
   0:	b119      	cbz	r1, a <ADC_SoftwareStartConvCmd+0xa>
D:\STM32\Program\1.11_Odchudzanie\um0427\FWLib\library\src/stm32f10x_adc.c:462
   2:	6883      	ldr	r3, [r0, #8]
   4:	f443 03a0 	orr.w	r3, r3, #5242880	; 0x500000
   8:	e002      	b.n	10 <ADC_SoftwareStartConvCmd+0x10>
D:\STM32\Program\1.11_Odchudzanie\um0427\FWLib\library\src/stm32f10x_adc.c:468
   a:	6883      	ldr	r3, [r0, #8]
   c:	f423 03a0 	bic.w	r3, r3, #5242880	; 0x500000
  10:	6083      	str	r3, [r0, #8]
D:\STM32\Program\1.11_Odchudzanie\um0427\FWLib\library\src/stm32f10x_adc.c:470
  12:	4770      	bx	lr
Disassembly of section .text.ADC_GetSoftwareStartConvStatus:

00000000 <ADC_GetSoftwareStartConvStatus>:
ADC_GetSoftwareStartConvStatus():
D:\STM32\Program\1.11_Odchudzanie\um0427\FWLib\library\src/stm32f10x_adc.c:487
   0:	6880      	ldr	r0, [r0, #8]
D:\STM32\Program\1.11_Odchudzanie\um0427\FWLib\library\src/stm32f10x_adc.c:500
   2:	f3c0 5080 	ubfx	r0, r0, #22, #1
   6:	4770      	bx	lr
Disassembly of section .text.ADC_DiscModeChannelCountConfig:

00000000 <ADC_DiscModeChannelCountConfig>:
ADC_DiscModeChannelCountConfig():
D:\STM32\Program\1.11_Odchudzanie\um0427\FWLib\library\src/stm32f10x_adc.c:522
   0:	6843      	ldr	r3, [r0, #4]
D:\STM32\Program\1.11_Odchudzanie\um0427\FWLib\library\src/stm32f10x_adc.c:527
   2:	3901      	subs	r1, #1
D:\STM32\Program\1.11_Odchudzanie\um0427\FWLib\library\src/stm32f10x_adc.c:524
   4:	f423 4360 	bic.w	r3, r3, #57344	; 0xe000
D:\STM32\Program\1.11_Odchudzanie\um0427\FWLib\library\src/stm32f10x_adc.c:527
   8:	ea43 3341 	orr.w	r3, r3, r1, lsl #13
D:\STM32\Program\1.11_Odchudzanie\um0427\FWLib\library\src/stm32f10x_adc.c:529
   c:	6043      	str	r3, [r0, #4]
D:\STM32\Program\1.11_Odchudzanie\um0427\FWLib\library\src/stm32f10x_adc.c:530
   e:	4770      	bx	lr
Disassembly of section .text.ADC_DiscModeCmd:

00000000 <ADC_DiscModeCmd>:
ADC_DiscModeCmd():
D:\STM32\Program\1.11_Odchudzanie\um0427\FWLib\library\src/stm32f10x_adc.c:549
   0:	b119      	cbz	r1, a <ADC_DiscModeCmd+0xa>
D:\STM32\Program\1.11_Odchudzanie\um0427\FWLib\library\src/stm32f10x_adc.c:552
   2:	6843      	ldr	r3, [r0, #4]
   4:	f443 6300 	orr.w	r3, r3, #2048	; 0x800
   8:	e002      	b.n	10 <ADC_DiscModeCmd+0x10>
D:\STM32\Program\1.11_Odchudzanie\um0427\FWLib\library\src/stm32f10x_adc.c:557
   a:	6843      	ldr	r3, [r0, #4]
   c:	f423 6300 	bic.w	r3, r3, #2048	; 0x800
  10:	6043      	str	r3, [r0, #4]
D:\STM32\Program\1.11_Odchudzanie\um0427\FWLib\library\src/stm32f10x_adc.c:559
  12:	4770      	bx	lr
Disassembly of section .text.ADC_RegularChannelConfig:

00000000 <ADC_RegularChannelConfig>:
ADC_RegularChannelConfig():
D:\STM32\Program\1.11_Odchudzanie\um0427\FWLib\library\src/stm32f10x_adc.c:613
   0:	2909      	cmp	r1, #9
D:\STM32\Program\1.11_Odchudzanie\um0427\FWLib\library\src/stm32f10x_adc.c:603
   2:	b510      	push	{r4, lr}
   4:	468c      	mov	ip, r1
   6:	4696      	mov	lr, r2
   8:	461c      	mov	r4, r3
D:\STM32\Program\1.11_Odchudzanie\um0427\FWLib\library\src/stm32f10x_adc.c:613
   a:	d90d      	bls.n	28 <ADC_RegularChannelConfig+0x28>
D:\STM32\Program\1.11_Odchudzanie\um0427\FWLib\library\src/stm32f10x_adc.c:618
   c:	2203      	movs	r2, #3
   e:	fb0c f202 	mul.w	r2, ip, r2
D:\STM32\Program\1.11_Odchudzanie\um0427\FWLib\library\src/stm32f10x_adc.c:620
  12:	2307      	movs	r3, #7
D:\STM32\Program\1.11_Odchudzanie\um0427\FWLib\library\src/stm32f10x_adc.c:618
  14:	3a1e      	subs	r2, #30
D:\STM32\Program\1.11_Odchudzanie\um0427\FWLib\library\src/stm32f10x_adc.c:620
  16:	4093      	lsls	r3, r2
D:\STM32\Program\1.11_Odchudzanie\um0427\FWLib\library\src/stm32f10x_adc.c:624
  18:	fa14 f202 	lsls.w	r2, r4, r2
D:\STM32\Program\1.11_Odchudzanie\um0427\FWLib\library\src/stm32f10x_adc.c:616
  1c:	68c1      	ldr	r1, [r0, #12]
D:\STM32\Program\1.11_Odchudzanie\um0427\FWLib\library\src/stm32f10x_adc.c:620
  1e:	ea21 0103 	bic.w	r1, r1, r3
D:\STM32\Program\1.11_Odchudzanie\um0427\FWLib\library\src/stm32f10x_adc.c:624
  22:	4311      	orrs	r1, r2
D:\STM32\Program\1.11_Odchudzanie\um0427\FWLib\library\src/stm32f10x_adc.c:626
  24:	60c1      	str	r1, [r0, #12]
  26:	e00b      	b.n	40 <ADC_RegularChannelConfig+0x40>
D:\STM32\Program\1.11_Odchudzanie\um0427\FWLib\library\src/stm32f10x_adc.c:633
  28:	2203      	movs	r2, #3
  2a:	fb0c f202 	mul.w	r2, ip, r2
D:\STM32\Program\1.11_Odchudzanie\um0427\FWLib\library\src/stm32f10x_adc.c:635
  2e:	2307      	movs	r3, #7
  30:	4093      	lsls	r3, r2
D:\STM32\Program\1.11_Odchudzanie\um0427\FWLib\library\src/stm32f10x_adc.c:639
  32:	fa14 f202 	lsls.w	r2, r4, r2
D:\STM32\Program\1.11_Odchudzanie\um0427\FWLib\library\src/stm32f10x_adc.c:631
  36:	6901      	ldr	r1, [r0, #16]
D:\STM32\Program\1.11_Odchudzanie\um0427\FWLib\library\src/stm32f10x_adc.c:635
  38:	ea21 0103 	bic.w	r1, r1, r3
D:\STM32\Program\1.11_Odchudzanie\um0427\FWLib\library\src/stm32f10x_adc.c:639
  3c:	4311      	orrs	r1, r2
D:\STM32\Program\1.11_Odchudzanie\um0427\FWLib\library\src/stm32f10x_adc.c:641
  3e:	6101      	str	r1, [r0, #16]
D:\STM32\Program\1.11_Odchudzanie\um0427\FWLib\library\src/stm32f10x_adc.c:644
  40:	f1be 0f06 	cmp.w	lr, #6	; 0x6
  44:	d80d      	bhi.n	62 <ADC_RegularChannelConfig+0x62>
D:\STM32\Program\1.11_Odchudzanie\um0427\FWLib\library\src/stm32f10x_adc.c:649
  46:	2205      	movs	r2, #5
  48:	fb0e f202 	mul.w	r2, lr, r2
D:\STM32\Program\1.11_Odchudzanie\um0427\FWLib\library\src/stm32f10x_adc.c:651
  4c:	231f      	movs	r3, #31
D:\STM32\Program\1.11_Odchudzanie\um0427\FWLib\library\src/stm32f10x_adc.c:649
  4e:	3a05      	subs	r2, #5
D:\STM32\Program\1.11_Odchudzanie\um0427\FWLib\library\src/stm32f10x_adc.c:651
  50:	4093      	lsls	r3, r2
D:\STM32\Program\1.11_Odchudzanie\um0427\FWLib\library\src/stm32f10x_adc.c:655
  52:	fa0c f202 	lsl.w	r2, ip, r2
D:\STM32\Program\1.11_Odchudzanie\um0427\FWLib\library\src/stm32f10x_adc.c:647
  56:	6b41      	ldr	r1, [r0, #52]
D:\STM32\Program\1.11_Odchudzanie\um0427\FWLib\library\src/stm32f10x_adc.c:651
  58:	ea21 0103 	bic.w	r1, r1, r3
D:\STM32\Program\1.11_Odchudzanie\um0427\FWLib\library\src/stm32f10x_adc.c:655
  5c:	4311      	orrs	r1, r2
D:\STM32\Program\1.11_Odchudzanie\um0427\FWLib\library\src/stm32f10x_adc.c:657
  5e:	6341      	str	r1, [r0, #52]
  60:	e01d      	b.n	9e <ADC_RegularChannelConfig+0x9e>
D:\STM32\Program\1.11_Odchudzanie\um0427\FWLib\library\src/stm32f10x_adc.c:660
  62:	f1be 0f0c 	cmp.w	lr, #12	; 0xc
  66:	d80d      	bhi.n	84 <ADC_RegularChannelConfig+0x84>
D:\STM32\Program\1.11_Odchudzanie\um0427\FWLib\library\src/stm32f10x_adc.c:665
  68:	2205      	movs	r2, #5
  6a:	fb0e f202 	mul.w	r2, lr, r2
D:\STM32\Program\1.11_Odchudzanie\um0427\FWLib\library\src/stm32f10x_adc.c:667
  6e:	231f      	movs	r3, #31
D:\STM32\Program\1.11_Odchudzanie\um0427\FWLib\library\src/stm32f10x_adc.c:665
  70:	3a23      	subs	r2, #35
D:\STM32\Program\1.11_Odchudzanie\um0427\FWLib\library\src/stm32f10x_adc.c:667
  72:	4093      	lsls	r3, r2
D:\STM32\Program\1.11_Odchudzanie\um0427\FWLib\library\src/stm32f10x_adc.c:671
  74:	fa0c f202 	lsl.w	r2, ip, r2
D:\STM32\Program\1.11_Odchudzanie\um0427\FWLib\library\src/stm32f10x_adc.c:663
  78:	6b01      	ldr	r1, [r0, #48]
D:\STM32\Program\1.11_Odchudzanie\um0427\FWLib\library\src/stm32f10x_adc.c:667
  7a:	ea21 0103 	bic.w	r1, r1, r3
D:\STM32\Program\1.11_Odchudzanie\um0427\FWLib\library\src/stm32f10x_adc.c:671
  7e:	4311      	orrs	r1, r2
D:\STM32\Program\1.11_Odchudzanie\um0427\FWLib\library\src/stm32f10x_adc.c:673
  80:	6301      	str	r1, [r0, #48]
  82:	e00c      	b.n	9e <ADC_RegularChannelConfig+0x9e>
D:\STM32\Program\1.11_Odchudzanie\um0427\FWLib\library\src/stm32f10x_adc.c:681
  84:	2205      	movs	r2, #5
  86:	fb0e f202 	mul.w	r2, lr, r2
D:\STM32\Program\1.11_Odchudzanie\um0427\FWLib\library\src/stm32f10x_adc.c:683
  8a:	231f      	movs	r3, #31
D:\STM32\Program\1.11_Odchudzanie\um0427\FWLib\library\src/stm32f10x_adc.c:681
  8c:	3a41      	subs	r2, #65
D:\STM32\Program\1.11_Odchudzanie\um0427\FWLib\library\src/stm32f10x_adc.c:683
  8e:	4093      	lsls	r3, r2
D:\STM32\Program\1.11_Odchudzanie\um0427\FWLib\library\src/stm32f10x_adc.c:687
  90:	fa0c f202 	lsl.w	r2, ip, r2
D:\STM32\Program\1.11_Odchudzanie\um0427\FWLib\library\src/stm32f10x_adc.c:679
  94:	6ac1      	ldr	r1, [r0, #44]
D:\STM32\Program\1.11_Odchudzanie\um0427\FWLib\library\src/stm32f10x_adc.c:683
  96:	ea21 0103 	bic.w	r1, r1, r3
D:\STM32\Program\1.11_Odchudzanie\um0427\FWLib\library\src/stm32f10x_adc.c:687
  9a:	4311      	orrs	r1, r2
D:\STM32\Program\1.11_Odchudzanie\um0427\FWLib\library\src/stm32f10x_adc.c:689
  9c:	62c1      	str	r1, [r0, #44]
D:\STM32\Program\1.11_Odchudzanie\um0427\FWLib\library\src/stm32f10x_adc.c:691
  9e:	bd10      	pop	{r4, pc}
Disassembly of section .text.ADC_ExternalTrigConvCmd:

00000000 <ADC_ExternalTrigConvCmd>:
ADC_ExternalTrigConvCmd():
D:\STM32\Program\1.11_Odchudzanie\um0427\FWLib\library\src/stm32f10x_adc.c:709
   0:	b119      	cbz	r1, a <ADC_ExternalTrigConvCmd+0xa>
D:\STM32\Program\1.11_Odchudzanie\um0427\FWLib\library\src/stm32f10x_adc.c:712
   2:	6883      	ldr	r3, [r0, #8]
   4:	f443 1380 	orr.w	r3, r3, #1048576	; 0x100000
   8:	e002      	b.n	10 <ADC_ExternalTrigConvCmd+0x10>
D:\STM32\Program\1.11_Odchudzanie\um0427\FWLib\library\src/stm32f10x_adc.c:717
   a:	6883      	ldr	r3, [r0, #8]
   c:	f423 1380 	bic.w	r3, r3, #1048576	; 0x100000
  10:	6083      	str	r3, [r0, #8]
D:\STM32\Program\1.11_Odchudzanie\um0427\FWLib\library\src/stm32f10x_adc.c:719
  12:	4770      	bx	lr
Disassembly of section .text.ADC_GetConversionValue:

00000000 <ADC_GetConversionValue>:
ADC_GetConversionValue():
D:\STM32\Program\1.11_Odchudzanie\um0427\FWLib\library\src/stm32f10x_adc.c:734
   0:	6cc0      	ldr	r0, [r0, #76]
D:\STM32\Program\1.11_Odchudzanie\um0427\FWLib\library\src/stm32f10x_adc.c:735
   2:	b280      	uxth	r0, r0
   4:	4770      	bx	lr
   6:	46c0      	nop			(mov r8, r8)
Disassembly of section .text.ADC_GetDualModeConversionValue:

00000000 <ADC_GetDualModeConversionValue>:
ADC_GetDualModeConversionValue():
D:\STM32\Program\1.11_Odchudzanie\um0427\FWLib\library\src/stm32f10x_adc.c:746
   0:	4b01      	ldr	r3, [pc, #4]	(8 <ADC_GetDualModeConversionValue+0x8>)
   2:	6818      	ldr	r0, [r3, #0]
D:\STM32\Program\1.11_Odchudzanie\um0427\FWLib\library\src/stm32f10x_adc.c:747
   4:	4770      	bx	lr
   6:	46c0      	nop			(mov r8, r8)
   8:	4001244c 	.word	0x4001244c
Disassembly of section .text.ADC_AutoInjectedConvCmd:

00000000 <ADC_AutoInjectedConvCmd>:
ADC_AutoInjectedConvCmd():
D:\STM32\Program\1.11_Odchudzanie\um0427\FWLib\library\src/stm32f10x_adc.c:766
   0:	b119      	cbz	r1, a <ADC_AutoInjectedConvCmd+0xa>
D:\STM32\Program\1.11_Odchudzanie\um0427\FWLib\library\src/stm32f10x_adc.c:769
   2:	6843      	ldr	r3, [r0, #4]
   4:	f443 6380 	orr.w	r3, r3, #1024	; 0x400
   8:	e002      	b.n	10 <ADC_AutoInjectedConvCmd+0x10>
D:\STM32\Program\1.11_Odchudzanie\um0427\FWLib\library\src/stm32f10x_adc.c:774
   a:	6843      	ldr	r3, [r0, #4]
   c:	f423 6380 	bic.w	r3, r3, #1024	; 0x400
  10:	6043      	str	r3, [r0, #4]
D:\STM32\Program\1.11_Odchudzanie\um0427\FWLib\library\src/stm32f10x_adc.c:776
  12:	4770      	bx	lr
Disassembly of section .text.ADC_InjectedDiscModeCmd:

00000000 <ADC_InjectedDiscModeCmd>:
ADC_InjectedDiscModeCmd():
D:\STM32\Program\1.11_Odchudzanie\um0427\FWLib\library\src/stm32f10x_adc.c:795
   0:	b119      	cbz	r1, a <ADC_InjectedDiscModeCmd+0xa>
D:\STM32\Program\1.11_Odchudzanie\um0427\FWLib\library\src/stm32f10x_adc.c:798
   2:	6843      	ldr	r3, [r0, #4]
   4:	f443 5380 	orr.w	r3, r3, #4096	; 0x1000
   8:	e002      	b.n	10 <ADC_InjectedDiscModeCmd+0x10>
D:\STM32\Program\1.11_Odchudzanie\um0427\FWLib\library\src/stm32f10x_adc.c:803
   a:	6843      	ldr	r3, [r0, #4]
   c:	f423 5380 	bic.w	r3, r3, #4096	; 0x1000
  10:	6043      	str	r3, [r0, #4]
D:\STM32\Program\1.11_Odchudzanie\um0427\FWLib\library\src/stm32f10x_adc.c:805
  12:	4770      	bx	lr
Disassembly of section .text.ADC_ExternalTrigInjectedConvConfig:

00000000 <ADC_ExternalTrigInjectedConvConfig>:
ADC_ExternalTrigInjectedConvConfig():
D:\STM32\Program\1.11_Odchudzanie\um0427\FWLib\library\src/stm32f10x_adc.c:854
   0:	6883      	ldr	r3, [r0, #8]
D:\STM32\Program\1.11_Odchudzanie\um0427\FWLib\library\src/stm32f10x_adc.c:856
   2:	f423 43e0 	bic.w	r3, r3, #28672	; 0x7000
D:\STM32\Program\1.11_Odchudzanie\um0427\FWLib\library\src/stm32f10x_adc.c:858
   6:	4319      	orrs	r1, r3
D:\STM32\Program\1.11_Odchudzanie\um0427\FWLib\library\src/stm32f10x_adc.c:860
   8:	6081      	str	r1, [r0, #8]
D:\STM32\Program\1.11_Odchudzanie\um0427\FWLib\library\src/stm32f10x_adc.c:861
   a:	4770      	bx	lr
Disassembly of section .text.ADC_ExternalTrigInjectedConvCmd:

00000000 <ADC_ExternalTrigInjectedConvCmd>:
ADC_ExternalTrigInjectedConvCmd():
D:\STM32\Program\1.11_Odchudzanie\um0427\FWLib\library\src/stm32f10x_adc.c:880
   0:	b119      	cbz	r1, a <ADC_ExternalTrigInjectedConvCmd+0xa>
D:\STM32\Program\1.11_Odchudzanie\um0427\FWLib\library\src/stm32f10x_adc.c:883
   2:	6883      	ldr	r3, [r0, #8]
   4:	f443 4300 	orr.w	r3, r3, #32768	; 0x8000
   8:	e002      	b.n	10 <ADC_ExternalTrigInjectedConvCmd+0x10>
D:\STM32\Program\1.11_Odchudzanie\um0427\FWLib\library\src/stm32f10x_adc.c:888
   a:	6883      	ldr	r3, [r0, #8]
   c:	f423 4300 	bic.w	r3, r3, #32768	; 0x8000
  10:	6083      	str	r3, [r0, #8]
D:\STM32\Program\1.11_Odchudzanie\um0427\FWLib\library\src/stm32f10x_adc.c:890
  12:	4770      	bx	lr
Disassembly of section .text.ADC_SoftwareStartInjectedConvCmd:

00000000 <ADC_SoftwareStartInjectedConvCmd>:
ADC_SoftwareStartInjectedConvCmd():
D:\STM32\Program\1.11_Odchudzanie\um0427\FWLib\library\src/stm32f10x_adc.c:909
   0:	b119      	cbz	r1, a <ADC_SoftwareStartInjectedConvCmd+0xa>
D:\STM32\Program\1.11_Odchudzanie\um0427\FWLib\library\src/stm32f10x_adc.c:913
   2:	6883      	ldr	r3, [r0, #8]
   4:	f443 1302 	orr.w	r3, r3, #2129920	; 0x208000
   8:	e002      	b.n	10 <ADC_SoftwareStartInjectedConvCmd+0x10>
D:\STM32\Program\1.11_Odchudzanie\um0427\FWLib\library\src/stm32f10x_adc.c:919
   a:	6883      	ldr	r3, [r0, #8]
   c:	f423 1302 	bic.w	r3, r3, #2129920	; 0x208000
  10:	6083      	str	r3, [r0, #8]
D:\STM32\Program\1.11_Odchudzanie\um0427\FWLib\library\src/stm32f10x_adc.c:921
  12:	4770      	bx	lr
Disassembly of section .text.ADC_GetSoftwareStartInjectedConvCmdStatus:

00000000 <ADC_GetSoftwareStartInjectedConvCmdStatus>:
ADC_GetSoftwareStartInjectedConvCmdStatus():
D:\STM32\Program\1.11_Odchudzanie\um0427\FWLib\library\src/stm32f10x_adc.c:938
   0:	6880      	ldr	r0, [r0, #8]
D:\STM32\Program\1.11_Odchudzanie\um0427\FWLib\library\src/stm32f10x_adc.c:951
   2:	f3c0 5040 	ubfx	r0, r0, #21, #1
   6:	4770      	bx	lr
Disassembly of section .text.ADC_InjectedChannelConfig:

00000000 <ADC_InjectedChannelConfig>:
ADC_InjectedChannelConfig():
D:\STM32\Program\1.11_Odchudzanie\um0427\FWLib\library\src/stm32f10x_adc.c:1005
   0:	2909      	cmp	r1, #9
D:\STM32\Program\1.11_Odchudzanie\um0427\FWLib\library\src/stm32f10x_adc.c:995
   2:	b510      	push	{r4, lr}
   4:	469c      	mov	ip, r3
   6:	468e      	mov	lr, r1
   8:	4614      	mov	r4, r2
D:\STM32\Program\1.11_Odchudzanie\um0427\FWLib\library\src/stm32f10x_adc.c:1005
   a:	d90d      	bls.n	28 <ADC_InjectedChannelConfig+0x28>
D:\STM32\Program\1.11_Odchudzanie\um0427\FWLib\library\src/stm32f10x_adc.c:1010
   c:	2203      	movs	r2, #3
   e:	fb0e f202 	mul.w	r2, lr, r2
D:\STM32\Program\1.11_Odchudzanie\um0427\FWLib\library\src/stm32f10x_adc.c:1012
  12:	2307      	movs	r3, #7
D:\STM32\Program\1.11_Odchudzanie\um0427\FWLib\library\src/stm32f10x_adc.c:1010
  14:	3a1e      	subs	r2, #30
D:\STM32\Program\1.11_Odchudzanie\um0427\FWLib\library\src/stm32f10x_adc.c:1012
  16:	4093      	lsls	r3, r2
D:\STM32\Program\1.11_Odchudzanie\um0427\FWLib\library\src/stm32f10x_adc.c:1016
  18:	fa0c f202 	lsl.w	r2, ip, r2
D:\STM32\Program\1.11_Odchudzanie\um0427\FWLib\library\src/stm32f10x_adc.c:1008
  1c:	68c1      	ldr	r1, [r0, #12]
D:\STM32\Program\1.11_Odchudzanie\um0427\FWLib\library\src/stm32f10x_adc.c:1012
  1e:	ea21 0103 	bic.w	r1, r1, r3
D:\STM32\Program\1.11_Odchudzanie\um0427\FWLib\library\src/stm32f10x_adc.c:1016
  22:	4311      	orrs	r1, r2
D:\STM32\Program\1.11_Odchudzanie\um0427\FWLib\library\src/stm32f10x_adc.c:1018
  24:	60c1      	str	r1, [r0, #12]
  26:	e00b      	b.n	40 <ADC_InjectedChannelConfig+0x40>
D:\STM32\Program\1.11_Odchudzanie\um0427\FWLib\library\src/stm32f10x_adc.c:1025
  28:	2203      	movs	r2, #3
  2a:	fb0e f202 	mul.w	r2, lr, r2
D:\STM32\Program\1.11_Odchudzanie\um0427\FWLib\library\src/stm32f10x_adc.c:1027
  2e:	2307      	movs	r3, #7
  30:	4093      	lsls	r3, r2
D:\STM32\Program\1.11_Odchudzanie\um0427\FWLib\library\src/stm32f10x_adc.c:1031
  32:	fa0c f202 	lsl.w	r2, ip, r2
D:\STM32\Program\1.11_Odchudzanie\um0427\FWLib\library\src/stm32f10x_adc.c:1023
  36:	6901      	ldr	r1, [r0, #16]
D:\STM32\Program\1.11_Odchudzanie\um0427\FWLib\library\src/stm32f10x_adc.c:1027
  38:	ea21 0103 	bic.w	r1, r1, r3
D:\STM32\Program\1.11_Odchudzanie\um0427\FWLib\library\src/stm32f10x_adc.c:1031
  3c:	4311      	orrs	r1, r2
D:\STM32\Program\1.11_Odchudzanie\um0427\FWLib\library\src/stm32f10x_adc.c:1033
  3e:	6101      	str	r1, [r0, #16]
D:\STM32\Program\1.11_Odchudzanie\um0427\FWLib\library\src/stm32f10x_adc.c:1038
  40:	6b81      	ldr	r1, [r0, #56]
D:\STM32\Program\1.11_Odchudzanie\um0427\FWLib\library\src/stm32f10x_adc.c:1042
  42:	2305      	movs	r3, #5
  44:	f3c1 5201 	ubfx	r2, r1, #20, #2
  48:	1aa2      	subs	r2, r4, r2
  4a:	3202      	adds	r2, #2
  4c:	b2d2      	uxtb	r2, r2
  4e:	fb02 f203 	mul.w	r2, r2, r3
D:\STM32\Program\1.11_Odchudzanie\um0427\FWLib\library\src/stm32f10x_adc.c:1044
  52:	331a      	adds	r3, #26
  54:	4093      	lsls	r3, r2
D:\STM32\Program\1.11_Odchudzanie\um0427\FWLib\library\src/stm32f10x_adc.c:1048
  56:	fa0e f202 	lsl.w	r2, lr, r2
D:\STM32\Program\1.11_Odchudzanie\um0427\FWLib\library\src/stm32f10x_adc.c:1044
  5a:	ea21 0103 	bic.w	r1, r1, r3
D:\STM32\Program\1.11_Odchudzanie\um0427\FWLib\library\src/stm32f10x_adc.c:1048
  5e:	4311      	orrs	r1, r2
D:\STM32\Program\1.11_Odchudzanie\um0427\FWLib\library\src/stm32f10x_adc.c:1050
  60:	6381      	str	r1, [r0, #56]
D:\STM32\Program\1.11_Odchudzanie\um0427\FWLib\library\src/stm32f10x_adc.c:1051
  62:	bd10      	pop	{r4, pc}
Disassembly of section .text.ADC_InjectedSequencerLengthConfig:

00000000 <ADC_InjectedSequencerLengthConfig>:
ADC_InjectedSequencerLengthConfig():
D:\STM32\Program\1.11_Odchudzanie\um0427\FWLib\library\src/stm32f10x_adc.c:1072
   0:	6b83      	ldr	r3, [r0, #56]
D:\STM32\Program\1.11_Odchudzanie\um0427\FWLib\library\src/stm32f10x_adc.c:1077
   2:	3901      	subs	r1, #1
D:\STM32\Program\1.11_Odchudzanie\um0427\FWLib\library\src/stm32f10x_adc.c:1074
   4:	f423 1340 	bic.w	r3, r3, #3145728	; 0x300000
D:\STM32\Program\1.11_Odchudzanie\um0427\FWLib\library\src/stm32f10x_adc.c:1077
   8:	ea43 5301 	orr.w	r3, r3, r1, lsl #20
D:\STM32\Program\1.11_Odchudzanie\um0427\FWLib\library\src/stm32f10x_adc.c:1079
   c:	6383      	str	r3, [r0, #56]
D:\STM32\Program\1.11_Odchudzanie\um0427\FWLib\library\src/stm32f10x_adc.c:1080
   e:	4770      	bx	lr
Disassembly of section .text.ADC_SetInjectedOffset:

00000000 <ADC_SetInjectedOffset>:
ADC_SetInjectedOffset():
D:\STM32\Program\1.11_Odchudzanie\um0427\FWLib\library\src/stm32f10x_adc.c:1099
   0:	b082      	sub	sp, #8
D:\STM32\Program\1.11_Odchudzanie\um0427\FWLib\library\src/stm32f10x_adc.c:1106
   2:	500a      	str	r2, [r1, r0]
D:\STM32\Program\1.11_Odchudzanie\um0427\FWLib\library\src/stm32f10x_adc.c:1107
   4:	b002      	add	sp, #8
   6:	4770      	bx	lr
Disassembly of section .text.ADC_GetInjectedConversionValue:

00000000 <ADC_GetInjectedConversionValue>:
ADC_GetInjectedConversionValue():
D:\STM32\Program\1.11_Odchudzanie\um0427\FWLib\library\src/stm32f10x_adc.c:1129
   0:	3028      	adds	r0, #40
   2:	5840      	ldr	r0, [r0, r1]
D:\STM32\Program\1.11_Odchudzanie\um0427\FWLib\library\src/stm32f10x_adc.c:1123
   4:	b082      	sub	sp, #8
D:\STM32\Program\1.11_Odchudzanie\um0427\FWLib\library\src/stm32f10x_adc.c:1130
   6:	b280      	uxth	r0, r0
   8:	b002      	add	sp, #8
   a:	4770      	bx	lr
Disassembly of section .text.ADC_AnalogWatchdogCmd:

00000000 <ADC_AnalogWatchdogCmd>:
ADC_AnalogWatchdogCmd():
D:\STM32\Program\1.11_Odchudzanie\um0427\FWLib\library\src/stm32f10x_adc.c:1157
   0:	6843      	ldr	r3, [r0, #4]
   2:	f423 0340 	bic.w	r3, r3, #12582912	; 0xc00000
   6:	f423 7300 	bic.w	r3, r3, #512	; 0x200
D:\STM32\Program\1.11_Odchudzanie\um0427\FWLib\library\src/stm32f10x_adc.c:1169
   a:	4319      	orrs	r1, r3
D:\STM32\Program\1.11_Odchudzanie\um0427\FWLib\library\src/stm32f10x_adc.c:1171
   c:	6041      	str	r1, [r0, #4]
D:\STM32\Program\1.11_Odchudzanie\um0427\FWLib\library\src/stm32f10x_adc.c:1172
   e:	4770      	bx	lr
Disassembly of section .text.ADC_AnalogWatchdogThresholdsConfig:

00000000 <ADC_AnalogWatchdogThresholdsConfig>:
ADC_AnalogWatchdogThresholdsConfig():
D:\STM32\Program\1.11_Odchudzanie\um0427\FWLib\library\src/stm32f10x_adc.c:1194
   0:	6241      	str	r1, [r0, #36]
D:\STM32\Program\1.11_Odchudzanie\um0427\FWLib\library\src/stm32f10x_adc.c:1196
   2:	6282      	str	r2, [r0, #40]
D:\STM32\Program\1.11_Odchudzanie\um0427\FWLib\library\src/stm32f10x_adc.c:1197
   4:	4770      	bx	lr
   6:	46c0      	nop			(mov r8, r8)
Disassembly of section .text.ADC_AnalogWatchdogSingleChannelConfig:

00000000 <ADC_AnalogWatchdogSingleChannelConfig>:
ADC_AnalogWatchdogSingleChannelConfig():
D:\STM32\Program\1.11_Odchudzanie\um0427\FWLib\library\src/stm32f10x_adc.c:1228
   0:	6843      	ldr	r3, [r0, #4]
   2:	f023 031f 	bic.w	r3, r3, #31	; 0x1f
D:\STM32\Program\1.11_Odchudzanie\um0427\FWLib\library\src/stm32f10x_adc.c:1240
   6:	4319      	orrs	r1, r3
D:\STM32\Program\1.11_Odchudzanie\um0427\FWLib\library\src/stm32f10x_adc.c:1242
   8:	6041      	str	r1, [r0, #4]
D:\STM32\Program\1.11_Odchudzanie\um0427\FWLib\library\src/stm32f10x_adc.c:1243
   a:	4770      	bx	lr
Disassembly of section .text.ADC_TempSensorVrefintCmd:

00000000 <ADC_TempSensorVrefintCmd>:
ADC_TempSensorVrefintCmd():
D:\STM32\Program\1.11_Odchudzanie\um0427\FWLib\library\src/stm32f10x_adc.c:1254
   0:	b120      	cbz	r0, c <ADC_TempSensorVrefintCmd+0xc>
D:\STM32\Program\1.11_Odchudzanie\um0427\FWLib\library\src/stm32f10x_adc.c:1261
   2:	4a05      	ldr	r2, [pc, #20]	(18 <ADC_TempSensorVrefintCmd+0x18>)
   4:	6893      	ldr	r3, [r2, #8]
   6:	f443 0300 	orr.w	r3, r3, #8388608	; 0x800000
   a:	e003      	b.n	14 <ADC_TempSensorVrefintCmd+0x14>
D:\STM32\Program\1.11_Odchudzanie\um0427\FWLib\library\src/stm32f10x_adc.c:1266
   c:	4a02      	ldr	r2, [pc, #8]	(18 <ADC_TempSensorVrefintCmd+0x18>)
   e:	6893      	ldr	r3, [r2, #8]
  10:	f423 0300 	bic.w	r3, r3, #8388608	; 0x800000
  14:	6093      	str	r3, [r2, #8]
D:\STM32\Program\1.11_Odchudzanie\um0427\FWLib\library\src/stm32f10x_adc.c:1268
  16:	4770      	bx	lr
  18:	40012400 	.word	0x40012400
Disassembly of section .text.ADC_GetFlagStatus:

00000000 <ADC_GetFlagStatus>:
ADC_GetFlagStatus():
D:\STM32\Program\1.11_Odchudzanie\um0427\FWLib\library\src/stm32f10x_adc.c:1293
   0:	6803      	ldr	r3, [r0, #0]
   2:	4219      	tst	r1, r3
D:\STM32\Program\1.11_Odchudzanie\um0427\FWLib\library\src/stm32f10x_adc.c:1306
   4:	bf0c      	ite	eq
   6:	2000      	moveq	r0, #0
   8:	2001      	movne	r0, #1
   a:	4770      	bx	lr
Disassembly of section .text.ADC_ClearFlag:

00000000 <ADC_ClearFlag>:
ADC_ClearFlag():
D:\STM32\Program\1.11_Odchudzanie\um0427\FWLib\library\src/stm32f10x_adc.c:1323
   0:	43c9      	mvns	r1, r1
   2:	6001      	str	r1, [r0, #0]
D:\STM32\Program\1.11_Odchudzanie\um0427\FWLib\library\src/stm32f10x_adc.c:1330
   4:	4770      	bx	lr
   6:	46c0      	nop			(mov r8, r8)
Disassembly of section .text.ADC_GetITStatus:

00000000 <ADC_GetITStatus>:
ADC_GetITStatus():
D:\STM32\Program\1.11_Odchudzanie\um0427\FWLib\library\src/stm32f10x_adc.c:1345
   0:	6842      	ldr	r2, [r0, #4]
D:\STM32\Program\1.11_Odchudzanie\um0427\FWLib\library\src/stm32f10x_adc.c:1360
   2:	6803      	ldr	r3, [r0, #0]
D:\STM32\Program\1.11_Odchudzanie\um0427\FWLib\library\src/stm32f10x_adc.c:1345
   4:	ea13 2011 	ands.w	r0, r3, r1, lsr #8
   8:	d004      	beq.n	14 <ADC_GetITStatus+0x14>
   a:	b2cb      	uxtb	r3, r1
   c:	4213      	tst	r3, r2
   e:	bf0c      	ite	eq
  10:	2000      	moveq	r0, #0
  12:	2001      	movne	r0, #1
D:\STM32\Program\1.11_Odchudzanie\um0427\FWLib\library\src/stm32f10x_adc.c:1373
  14:	4770      	bx	lr
  16:	46c0      	nop			(mov r8, r8)
Disassembly of section .text.ADC_ClearITPendingBit:

00000000 <ADC_ClearITPendingBit>:
ADC_ClearITPendingBit():
D:\STM32\Program\1.11_Odchudzanie\um0427\FWLib\library\src/stm32f10x_adc.c:1388
   0:	ea6f 2111 	mvn.w	r1, r1, lsr #8
   4:	6001      	str	r1, [r0, #0]
D:\STM32\Program\1.11_Odchudzanie\um0427\FWLib\library\src/stm32f10x_adc.c:1400
   6:	4770      	bx	lr
Disassembly of section .text.ADC_DeInit:

00000000 <ADC_DeInit>:
ADC_DeInit():
D:\STM32\Program\1.11_Odchudzanie\um0427\FWLib\library\src/stm32f10x_adc.c:131
   0:	b507      	push	{r0, r1, r2, lr}
D:\STM32\Program\1.11_Odchudzanie\um0427\FWLib\library\src/stm32f10x_adc.c:135
   2:	4b13      	ldr	r3, [pc, #76]	(50 <ADC_DeInit+0x50>)
D:\STM32\Program\1.11_Odchudzanie\um0427\FWLib\library\src/stm32f10x_adc.c:131
   4:	9001      	str	r0, [sp, #4]
D:\STM32\Program\1.11_Odchudzanie\um0427\FWLib\library\src/stm32f10x_adc.c:135
   6:	4298      	cmp	r0, r3
   8:	d00f      	beq.n	2a <ADC_DeInit+0x2a>
   a:	f503 53a0 	add.w	r3, r3, #5120	; 0x1400
   e:	4298      	cmp	r0, r3
  10:	d013      	beq.n	3a <ADC_DeInit+0x3a>
  12:	f5a3 53c0 	sub.w	r3, r3, #6144	; 0x1800
  16:	4298      	cmp	r0, r3
  18:	d119      	bne.n	4e <ADC_DeInit+0x4e>
D:\STM32\Program\1.11_Odchudzanie\um0427\FWLib\library\src/stm32f10x_adc.c:139
  1a:	f44f 7000 	mov.w	r0, #512	; 0x200
  1e:	2101      	movs	r1, #1
  20:	f7ff fffe 	bl	0 <RCC_APB2PeriphResetCmd>
D:\STM32\Program\1.11_Odchudzanie\um0427\FWLib\library\src/stm32f10x_adc.c:141
  24:	f44f 7000 	mov.w	r0, #512	; 0x200
  28:	e00e      	b.n	48 <ADC_DeInit+0x48>
D:\STM32\Program\1.11_Odchudzanie\um0427\FWLib\library\src/stm32f10x_adc.c:146
  2a:	f44f 6080 	mov.w	r0, #1024	; 0x400
  2e:	2101      	movs	r1, #1
  30:	f7ff fffe 	bl	0 <RCC_APB2PeriphResetCmd>
D:\STM32\Program\1.11_Odchudzanie\um0427\FWLib\library\src/stm32f10x_adc.c:148
  34:	f44f 6080 	mov.w	r0, #1024	; 0x400
  38:	e006      	b.n	48 <ADC_DeInit+0x48>
D:\STM32\Program\1.11_Odchudzanie\um0427\FWLib\library\src/stm32f10x_adc.c:153
  3a:	f44f 4000 	mov.w	r0, #32768	; 0x8000
  3e:	2101      	movs	r1, #1
  40:	f7ff fffe 	bl	0 <RCC_APB2PeriphResetCmd>
D:\STM32\Program\1.11_Odchudzanie\um0427\FWLib\library\src/stm32f10x_adc.c:155
  44:	f44f 4000 	mov.w	r0, #32768	; 0x8000
  48:	2100      	movs	r1, #0
  4a:	f7ff fffe 	bl	0 <RCC_APB2PeriphResetCmd>
D:\STM32\Program\1.11_Odchudzanie\um0427\FWLib\library\src/stm32f10x_adc.c:161
  4e:	bd0e      	pop	{r1, r2, r3, pc}
  50:	40012800 	.word	0x40012800
